:1000000023C032C031C030C02FC0ACC02DC02CC006
:100010002BC02AC029C028C027C026C025C0010285
:100020000000040000000000000000003800000094
:100030000000370002020202020202020202010272
:10004000040810202004100811241FBECFE5D2E0C0
:10005000DEBFCDBF20E0A0E6B0E001C01D92A93612
:10006000B207E1F7C9D01CC1CBCF90E0FC01E25C44
:10007000FF4F24918C5C9F4FFC018491882399F061
:1000800090E0880F991FFC01E25DFF4FA591B491AC
:10009000FC01E85DFF4F859194918FB7F894EC9146
:1000A000E22BEC938FBF089590E0FC01E25EFF4FDE
:1000B0003491FC01E25CFF4F2491FC01EC5CFF4FAA
:1000C000E491EE23B9F0332329F0323001F198F4B2
:1000D0003130C9F0F0E0EE0FFF1FE85DFF4FA59152
:1000E000B4918FB7F894EC91611114C020952E2330
:1000F0002C938FBF0895333011F0343059F78CB5FD
:100100008F7D8CBDE7CF8AB58F778ABDE3CF8AB567
:100110008F7DFBCF2E2BECCF3FB7F89480916500FD
:1001200090916600A0916700B091680022B708B670
:1001300001FE05C02F3F19F00196A11DB11D3FBF63
:10014000BA2FA92F982F8827BC01CD01620F711DEE
:10015000811D911D46E0660F771F881F991F4A95E4
:10016000D1F708951F920F920FB60F9211242F937B
:100170003F938F939F93AF93BF9380916100909132
:100180006200A0916300B09164003091600020E3B0
:10019000230F2D3758F54096A11DB11D2093600007
:1001A0008093610090936200A0936300B093640019
:1001B0008091650090916600A0916700B091680001
:1001C0000196A11DB11D8093650090936600A093D8
:1001D0006700B0936800BF91AF919F918F913F915D
:1001E0002F910F900FBE0F901F90189523EB230FA8
:1001F0004196A11DB11DD2CF78948AB582608ABD87
:100200008AB581608ABD83B7826083BF83B781600E
:1002100083BF89B7826089BF80B7826080BF329810
:10022000319A309A379A8CB580648CBD80E01DDF9E
:1002300081E01BDF00E010E0C0E061E08C2F34DFE4
:1002400060E081E08C2730DF67DF4B015C0180E9F3
:10025000C82EDD24D394E12CF12C5EDF68197909D6
:100260008A099B09683E734081059105B0F321E03E
:10027000C21AD108E108F10888EE880E83E0981EC2
:10028000A11CB11CC114D104E104F10431F7C13047
:1002900029F40115110581F2B3DECECFC1E0CDCF37
:0402A000F894FFCF00
:00000001FF
